:020000040000FA
:020000000828CE
:040008000B1116289A
:100010008B13A32033308500A8018519A80AB430BA
:1000200081008B168B17000000001328B43081006C
:100030002520302052303B2020083B2022083B2046
:100040003330850001303B200900A0018512051CDA
:100050002E280000A00F2728FF30A00085160800DA
:10006000A2010512851C39280000A20F3228FF309A
:10007000A20005160800281C3E287A28A300063096
:10008000A40005150000442845284628472848288C
:100090000000051100004C284D284E284F285028FC
:1000A00000000515000054285528562857285828C0
:1000B0000000051100005C285D285E285F2860288C
:1000C0000000051500006428652866286728682850
:1000D0000000051100006C286D286E286F28A4030D
:1000E000031D4128AF207428752876287728A30B94
:1000F00073280800A3000E30A40005150000802816
:10010000812882280511000085288628872800007C
:10011000051500008B288C288D28051100009028DB
:100120009128A403031D7D28AF209628972898289E
:100130000000A30B95280A30A50000000000000075
:10014000A50B9D2808008316FF2390000B30850027
:100150008730810083120730990085010800043040
:10016000A600B520A60BB12808000730A700A70BF2
:04017000B7280800A4
:02400E00843FED
:00000001FF
